:020000040000FA
:100000003430831690008312073099003F3085000A
:1000100083165230810095010E3085008312FA302C
:10002000BD20FA30BD20851D78283030A3002F3048
:100030002307A400CB2083169B01831205122308FB
:100040008400840A851C2728051D24283A280519C0
:1000500027282A280B1181010B1D312885184B28D0
:100060006628051D2C2801088000840A0408240243
:1000700003195F280B1181010B1D4128851C4B289A
:10008000662805193C2801088000840A0408240217
:1000900003195F282A280408A00023080402A100ED
:1000A0000130A10223088400210880003030A30021
:1000B000E5200516FA30BD20FA30BD201E280516B1
:1000C000FA30BD200512FA30BD205F280516323007
:1000D000BD200512FA30BD20FA30BD2005163230A1
:1000E000BD200512FA30BD20FA30BD2066287728E1
:1000F00083160A3085009B018312051585180511AA
:100100000630A200FA30BD20A20B822885123030C2
:1001100084000B21A0008000840A013E0319B82846
:100120000B218000840AA00B902830308400000846
:10013000A000840A05199E2805159F280511810134
:1001400000080102031DA028840AA00B9A280515A7
:1001500085180511FA30BD20FA30BD20FA30BD20D7
:100160008516FA30BD20FA30BD20FA30BD20862831
:10017000851683160E308500BC28A1006E30A000C5
:10018000000000000000000000000000A00BC028DC
:10019000A10BBE2808008030A000FF3083169A0013
:1001A0009B0183161C1555309D00AA309D009C14A0
:1001B0009C18D8281C111A081C141A06031DD128D3
:1001C0009B0A8312A00BD12808003030840000085D
:1001D000A000A00A83169A0083161C1555309D00B6
:1001E000AA309D009C149C18F3281C111A081C149A
:1001F0001A06031DEC288312840A000883169B0A42
:100200009A007F309B0503011B06831203195F28A8
:10021000A00BEC28080083161C141A089B0A8312F2
:1002200008002A0045006D0069006C0069006F003D
:100230002A002800320039002D00300035002D0042
:1002400030003700290000340034FF3FFF3FFF3FFC
:10025000FF3FFF3FFF3FFF3FFF3FFF3FFF3FFF3FAE
:10026000FF3FFF3FFF3FFF3FFF3FFF3FFF3FFF3F9E
:10027000FF3FFF3FFF3FFF3FFF3FFF3FFF3FFF3F8E
:10028000FF3FFF3FFF3FFF3FFF3FFF3FFF3FFF3F7E
:1042000019007A006100E9005E007C005E007C001D
:104210005E007C005D007C005D007C00CE007900CB
:104220006100790061007900610079006100790026
:1042300061007C0017007900610079006100E900ED
:104240005E007C005E007C005E007C005E007C0006
:10425000CF007800610079006100E9005E007C0019
:104260005E007C00190073006700E60061007800C2
:1042700061007600640079006100780061007500DB
:10428000D600750064007600640072006800750056
:104290006500720067007900170070006B006E0007
:1042A0006C00DF0068007200680071006900710036
:1042B00068007200D9006E006B006E006C00DF00B9
:1042C000680072006800710017006D006E00DF006A
:1042D00068006F006B007100680072006800720077
:1042E00068007100D9006B006E006C006E00DF008A
:1042F00068006F006B006E000100A600FF00FF0069
:02400E00843FED
:08400000FF3FFF3FFF3FFF3FC0
:0207FE000034C5
:00000001FF
